:100000000C94F6000C9415010C9415010C94150138
:100010000C9415010C9415010C9415010C94150108
:100020000C9415010C9415010C9417060C941501F1
:100030000C9415010C9415010C9415010C941501E8
:100040000C9415010C9415010C9415010C941501D8
:100050000C9415010C9415010C9415010C941501C8
:100060000C9415010C9415010C9415010C941501B8
:100070000C9415010C9415010C9415010C941501A8
:100080000C9415010C9415010C9415010C94150198
:100090000C9415010C941501002C2AE1080C110692
:1000A0001712160915101A14040B071C0F13050D4F
:1000B000180A191B0E1D002B363733342F303138F8
:1000C0001E1F20212223242526272D2E2835E2E05D
:1000D000504F52514B4E494C4A4D4648E539E3E7A3
:1000E0003A3B3C3D3E3F40414243444529291201B1
:1000F00000020000004000000200001001020301A5
:1001000009023B00020100C03209040000010300A3
:1001100002000921011000012234000705810308B3
:10012000000509040100010300010109210110007B
:1001300001223B00070582030800050C034F005411
:10014000004C004C0043002603430048004F00527F
:100150000044004900540045002000500052004F68
:100160000054004F0054005900500045000C03306B
:10017000002E0030002E003100040309040501099F
:1001800002A1010901A10005091901290315002592
:10019000017501950381027505950181010501092C
:1001A00030093109381581257F750895038106C00E
:1001B000C005010906A101050719E029E715002579
:1001C0000175019508810281011900296515002535
:1001D0006575089506810005081901290515002592
:1001E0000175019505910295039101C011241FBE6F
:1001F000CFEFD0E2DEBFCDBF11E0A0E0B1E0EEEC8A
:10020000F2E100E00BBF02C007900D92A430B107ED
:10021000D9F711E0A4E0B1E001C01D92A832B10706
:10022000E1F70E9468050C9466090C940000833085
:1002300039F5613069F0613028F0623079F063306F
:10024000F9F412C084E08093240189E791E011C0A1
:100250008CE0809324018BE391E00BC086E28093D5
:10026000240187E491E005C08CE0809324018DE6B1
:1002700091E0909326018093250181E090E008951C
:1002800080E090E00895CF93DF93CDB7DEB722975B
:100290000FB6F894DEBF0FBECDBF8091F100809302
:1002A00021018091F10080932201809121019091A0
:1002B0002201009719F0019781F406C084E380932E
:1002C00024018DE791E005C08BE38093240181EB4D
:1002D00091E090932601809325018091F10089831C
:1002E0008091F1008A838091E800877F8093E80005
:1002F00029813A818091240190E08217930770F45C
:100300008F739070892B11F441E001C040E0E091BF
:100310002501F0912601909124011AC02093240117
:10032000F5CF8091E80080FFFCCF30E00AC03F5F4E
:10033000292F2150313439F084918093F100319686
:10034000922F9923A1F78091E8008E7F8093E80097
:10035000992359F08091E80082FFE3CFF0932601C2
:10036000E09325019093240106C0F0932601E093C9
:100370002501109224018091E8008E7F8093E8008F
:100380008091E80082FD0BC0413029F48091E800A3
:100390008E7F8093E8008091E80082FFFCCF8091FF
:1003A000E8008B7F8093E8008091E8008F7780934E
:1003B000E80022960FB6F894DEBF0FBECDBFDF91E6
:1003C000CF9108958091E800877F8093E800809125
:1003D000E8008E7F8093E8008091E80082FFFCCFE8
:1003E0008091E8008B7F8093E8008091E8008F7710
:1003F0008093E8008091E8008E7F8093E800089564
:100400008091F1008091F1008091F10080932101B1
:100410008091F100809322018091E800877F809392
:10042000E8008091E8008E7F8093E8008091E800EA
:1004300080FFFCCF08958091F1008091F1008091C0
:10044000F100809321018091F1008093220180913D
:10045000E800877F8093E8008091E8008E7F80939A
:10046000E8008091E80080FFFCCF0895CF93DF93F0
:10047000CDB7DEB722970FB6F894DEBF0FBECDBF63
:100480008091F100809321018091F10080932201FD
:100490008091210190912201009719F0019781F438
:1004A00006C089E08093240182E191E005C089E0E3
:1004B000809324018BE291E09093260180932501A3
:1004C0008091F10089838091F1008A838091E80016
:1004D000877F8093E80029813A818091240190E010
:1004E0008217930770F48F739070892B11F441E099
:1004F00001C040E0E0912501F09126019091240196
:100500001AC020932401F5CF8091E80080FFFCCF32
:1005100030E00AC03F5F292F2150313439F08491F7
:100520008093F1003196922F9923A1F78091E800F2
:100530008E7F8093E800992359F08091E80082FF34
:10054000E3CFF0932601E09325019093240106C0A8
:10055000F0932601E0932501109224018091E80098
:100560008E7F8093E8008091E80082FD0BC04130CF
:1005700029F48091E8008E7F8093E8008091E80064
:1005800082FFFCCF8091E8008B7F8093E800809110
:10059000E8008F778093E80022960FB6F894DEBFCC
:1005A0000FBECDBFDF91CF9108958091F100809172
:1005B000F100693071F06A3089F06630A1F481325F
:1005C00029F0823281F40E9443010AC00E9436025F
:1005D00007C0823041F40E94E20102C00E941B0267
:1005E00081E090E0089580E090E008950F931F93DC
:1005F00009EE10E081E0F801808360E081EC0E9468
:100600009F0582E0F801808360E081EC0E949F05F5
:100610001F910F91089510921801109219011092D4
:100620001A0110921B0110921E01E2EEF0E080818F
:1006300084608083089580911E018F5F80931E01E6
:100640000895E0EEF0E080818160808308958091DC
:100650001E01833008F487C010921E011092180109
:100660001092190110921A0110921B010E94E403CA
:10067000482F882329F480910501882321F473C031
:100680008E3109F470C0642F70E09B012F703070C0
:100690002A30310531F480911A01815080931A017A
:1006A00025C02230310559F480911A018150809380
:1006B0001A01809119018F5F8093190120C02330A6
:1006C000310531F4809119018F5F809319011EC0AB
:1006D0002130310559F480911A018F5F80931A01FE
:1006E000809119018F5F8093190113C02530310566
:1006F00031F480911A018F5F80931A0117C0243062
:10070000310521F480911A018F5F09C02C30310529
:1007100041F02830310551F480911A0181508093C5
:100720001A0180911901815080931901CB018073C6
:1007300090708031910521F48091180181600CC086
:100740008032910521F480911801826005C0C09724
:1007500029F4809118018460809318014093050169
:1007600081E090E0089580E090E008958091060196
:10077000882349F180912301882329F10E942703CE
:10078000882309F181E08093E9008091E80085FFEA
:100790001AC0809118018093F10080911901809313
:1007A000F10080911A018093F10080911B018093E8
:1007B000F1008091E8008E7F8093E8008091E8004E
:1007C0008F778093E8000895CF93DF93CDB7DEB79E
:1007D00024970FB6F894DEBF0FBECDBF83B18095CE
:1007E000898383B180958A8383B180958B8383B11C
:1007F00080958C8320E030E0BE016F5F7F4F09C0A1
:1008000083B19370FB01E90FF11D809580832F5F09
:100810003F4F922F49818A81481791F78B81481762
:1008200079F78C81481761F740931001442329F42C
:1008300080910F018823F9F455C04E31E1F4809185
:100840000F018E31C1F080910601882359F481E0B7
:100850008093060184E690E090930101809300016B
:100860005C9A09C01092060184E690E09093010121
:10087000809300015C9890910F01242F2923291760
:1008800071F010920E0110920D0140930F018091B2
:100890000201882339F110920201892F21C0822F91
:1008A000842B821751F081E08093020110920E0197
:1008B00010920D0140930F0115C020910D01309150
:1008C0000E0180910001909101012817390738F439
:1008D0002F5F3F4F30930E0120930D0103C0842FF3
:1008E00090E002C080E090E024960FB6F894DEBF5E
:1008F0000FBECDBFDF91CF910895AC018AB1806F5B
:100900008AB920910B0130910C01CA019695879507
:100910002817390710F45C9A01C05C98C901019648
:1009200090930C0180930B018417950720F010928F
:100930000C0110920B010895AC018AB1806F8AB945
:100940002091090130910A01CA01969587952817CF
:10095000390710F45E9A01C05E98C9010196909320
:100960000A01809309018417950720F010920A016B
:1009700010920901089514B88FEF85B98AB1806F7C
:100980008AB910921E01E2EEF0E0808184608083DB
:100990000895282F882369F480910701803EF0F59F
:1009A0008823E1F1109207011092080180E090E0A5
:1009B0000895833EF1F0843E38F4813E91F0823E0A
:1009C000A0F4803E59F509C0853ED9F0853EA8F0D7
:1009D000863ED9F0873E11F51CC0809108018160E8
:1009E0001BC080910801826017C08091080184605B
:1009F00013C08091080188600FC080910801806158
:100A00000BC080910801806207C08091080180645A
:100A100003C08091080180688093080190910801CB
:100A2000992311F05D9A01C05D98293329F48091D2
:100A30000701893309F04E9A20930701892F90E02E
:100A4000089580910601882309F041C082E08093D7
:100A5000E9008091E80080FF3AC08091230188235B
:100A6000B1F18091E80080FFFCCF0E94E403809305
:100A70002001863510F010922001E0912001F0E075
:100A8000E856FF4FE491E093200182E08093E90073
:100A90008E2F0E94C9048093F1001092F100809182
:100AA00020018093F1001092F1001092F100109259
:100AB000F1001092F1001092F1008091E8008E7F19
:100AC0008093E8008091E8008F778093E800089594
:100AD000A89587EF84BFE0E6F0E08081886180839D
:100AE0001082E1E6F0E080E8808310820E946109D4
:100AF00080E090E0089513BE83B7856083BF88953A
:100B0000089513BE83B7816083BF8895089513BE8F
:100B100083B7836083BF8895089513BE83B78760CA
:100B200083BF8895089513BE83B78D6083BF889572
:100B3000089513BE83B78F6083BF88950895909101
:100B4000EB0091609093EB008093EC008091ED00BE
:100B50008270862B8093ED008091ED0082608093FF
:100B6000ED008091EE00992787FD90958827990FD9
:100B7000881F992708954091F40020E030E0822FEB
:100B800040FF02C090E008952F5F3F4F27303105AE
:100B900011F04695F4CF80E090E00895FB0180933A
:100BA000E90004C081918093F10041508091E800F8
:100BB00085FF02C04423B1F7842F90E00895FB0124
:100BC0008093E90004C08091F100819341508091AD
:100BD000E80085FF02C04423B1F7842F90E0089518
:100BE0008093E900EBEEF0E08081806280830895DD
:100BF0008091D8008F7B8093D8008091D90081FFAD
:100C00000EC01092E9008091EB0080FD08C01092A8
:100C1000E90060E382E00E949F0590E0089580E093
:100C200090E00895089578940E947B0508951F929E
:100C30000F920FB60F9211242F933F934F935F9310
:100C40006F937F938F939F93AF93BF93EF93FF9394
:100C50008091DA0080FF33C08091D80080FF2FC0E0
:100C60008EEF8093DA008091D90080FF19C081E077
:100C700080932701809111019091120182609093DD
:100C80001201809311018091E20088608093E2005C
:100C90000E940A098091E0008E7F8093E0000FC0DF
:100CA0000E942103109227011092230180911101CB
:100CB00090911201846090931201809311018091B0
:100CC000E10082FF09C08091E20082FF05C08BEF46
:100CD0008093E1000E941B038091E10080FF1FC010
:100CE0008091E20080FF1BC08EEF8093E100809135
:100CF000E20080618093E2008FEE8093E1008091BA
:100D0000D80080628093D8008091110190911201E7
:100D1000806290931201809311010E9413068091CA
:100D2000E10084FF1AC08091E20084FF16C0809128
:100D3000D8008F7D8093D8008FEE8093E100809162
:100D4000E2008F7E8093E200809111019091120168
:100D5000806490931201809311018091E10085FFDE
:100D60001AC08091E20085FF16C08091E2008F7E5C
:100D70008093E2008FED8093E1008091E2008F7D0F
:100D80008093E2008091110190911201806890930C
:100D90001201809311018091E10083FF12C08091C4
:100DA000E20083FF0EC087EF8093E1000E94F80508
:100DB00080911101909112019160909312018093A2
:100DC0001101FF91EF91BF91AF919F918F917F9111
:100DD0006F915F914F913F912F910F900FBE0F90A8
:100DE0001F9018950E9426090895E7EDF0E0808194
:100DF0008160808380818F7B808380818068808315
:100E00000E94F9080895CF93DF93CDB7DEB72297FC
:100E10000FB6F894DEBF0FBECDBF9091F100909356
:100E200017016091F1006630F9F0673068F46130C5
:100E300009F400C1613008F46AC1633009F433C1B8
:100E4000653009F0BEC1BCC0693009F4DAC06A304F
:100E500020F4683009F0B5C197C06A3009F499C12F
:100E60006B3009F0AEC19CC1903809F08BC0109274
:100E700013016091F1008091F100813019F082300E
:100E800089F406C082E1809324018EEE90E005C0D3
:100E90008BE38093240180E091E09093260180937E
:100EA000250105C00E941701882309F48FC1809194
:100EB000F1008091F1008091F10089838091F1002F
:100EC0008A838091E800877F8093E80029813A81B6
:100ED0008091240190E08217930758F48F739070EB
:100EE000892B21F481E08093130105C01092130136
:100EF00002C020932401E0912501F09126019091F8
:100F0000240117C08091E80080FFFCCF30E00AC0C8
:100F10003F5F292F2150313439F084918093F100C3
:100F20003196922F9923A1F78091E8008E7F8093CC
:100F3000E800992359F08091E80082FFE3CFF09315
:100F40002601E09325019093240106C0F093260129
:100F5000E0932501109224018091E80082FD10C1E8
:100F600080911301813049F48091E80080FFFCCF2B
:100F70008091E8008E7F8093E8008091E80082FFF6
:100F8000FCCFFEC066E008C19038C1F48091E80053
:100F9000877F8093E800809123018093F100809106
:100FA000E8008E7F8093E8008091E8008F7780933F
:100FB000E8008091E80082FFFCCFE2C068E0ECC06E
:100FC0009923E9F49091E3008091F1008F77907874
:100FD000892B8093E3008091E800877F8093E8006D
:100FE0008091E8008E7F8093E8008091E80080FF88
:100FF000FCCF8091E30080688093E300F1C065E05E
:10100000CBC09923A9F49091F100923008F0DEC092
:101010008091E800877F8093E8009093230180917E
:10102000E8008E7F8093E800892F0E94F602D8C0E6
:1010300069E0B2C09330A8F5992309F4C7C0913094
:1010400009F4C4C08091F1009091F100882309F067
:10105000BDC0E091F100EF77E093E9008091EB00F3
:1010600080FF50C0EE23B1F08091EB00806180934F
:10107000EB0081E090E00E2E02C0880F991F0A94C9
:10108000E2F78093EA001092EA008091EB0088601A
:101090008093EB001092E900F0E0EC5EFE4F1082CE
:1010A00028C061E079C0933080F5913009F48EC09A
:1010B000923009F095C08091F1009091F100882361
:1010C00009F084C0E091F100EF7709F47FC0E0936C
:1010D000E9008091EB0080FF15C08091EB008062F9
:1010E0008093EB001092E900F0E0EC5EFE4F81E0AF
:1010F00080838091E800877F8093E8008091E800FA
:101100008E7F6CC01092E90061C063E045C0892FFA
:101110008058833008F040C08091F1008091F10048
:10112000E091F100913861F0923891F0903809F037
:101130004DC08091E800877F8093E80081E013C074
:101140008091E800877F8093E8001092F1000DC045
:101150008091E800877F8093E800F0E0EF77F070FF
:10116000EC5EFE4F80818093F1001092F10080913F
:10117000E8008E7F8093E8008091E80082FFFCCF3A
:101180008091E8008B7F8093E8008091E8008F7762
:1011900025C09138D9F06AE0892F0E94D50220C07D
:1011A0009130F1F48091E800877F8093E80080918E
:1011B000E8008E7F8093E8008091E80080FD10C0F9
:1011C000FBCF892F0E94D502882351F48091EB0038
:1011D00080628093EB008091E800877F8093E80035
:1011E00022960FB6F894DEBF0FBECDBFDF91CF9130
:1011F00008957894E8EDF0E080818F768083808197
:101200008069808380818F7B8083808181608083FF
:10121000789408958EE089BD09B400FEFDCF8091D9
:10122000D8008F7D8093D8008091E2008160809308
:10123000E2008091E20088608093E2000E94F8055D
:101240008091E0008E7F8093E00008958091D90026
:1012500080FF09C080912701882329F481E08093D1
:1012600027010E940A09809111019091120190FFBB
:1012700010C080911101909112019E7F90931201F4
:101280008093110181E08093EA001092EA001092AD
:1012900023011092E9008091E80083FF02C00E94C0
:1012A0000307089508950E94F2060E94B6030E9463
:1012B0002105F9CF0E94F5060E940B030E94BB0492
:0E12C00008950E945A090E9453090895FFCF15
:0412CE0064000100B7
:00000001FF
